:100000000C943B040C9482040C9482040C9482049F
:100010000C9482040C9482040C9482040C94820448
:100020000C9482040C9482040C94A42B0C94762CD3
:100030000C94FF210C9482040C9482040C9482048E
:100040000C9482040C9482040C9482040C94820418
:100050000C9482040C9467220C9482040C94820405
:100060000C9482040C9482040C9482040C948204F8
:100070000C9482040C9482040C9482040C948204E8
:100080000C9482040C9482040C9482040C948204D8
:100090000C9482040C9482040C9482040C948204C8
:1000A0000C9482040C9482040C9482045F0764070D
:1000B0006E07620767076C076A07110813081E08B6
:1000C0001508170819081B081D082008220824080D
:1000D0002F08260828082A082C082E083108D017CF
:1000E000D0170A180A183F185F18CC19081AA11857
:1000F000081A51195119C419081A081A031A5E1955
:100100005E195E195E195E195E195E195E195E1937
:100110005E195E195E195E195E195E195E19701915
:100120007D1984198B199519971A971AA91AA91A62
:10013000A01AA91AA91AA91A971A971AA51AA91AD8
:10014000A91AA51AE32C0A2DFC2D0A2DFC2D562DDB
:10015000792DFC2DCF2DDE2D07634236B79BD8A716
:100160001A39685618AEBAAB558C1D3CB7CC5763DC
:10017000BD6DEDFD753EF6177231BF000000803F8A
:1001800005A84CCDB2D44EB93836A9020C50B9915D
:100190008688083CA6AAAA2ABE000000803F657295
:1001A000676F646F785F657A2F63663937393761B7
:1001B0003635653966323837666533353320402049
:1001C000302E352E3135362D31312D6738343761AB
:1001D0006465006572676F646F785F657A2F636628
:1001E00039373937613635653966323837666533C0
:1001F0003533204020302E352E3135362D31312DFE
:1002000067383437616465000000F0A135002B00C9
:1002100029623961500000001E00140004001D0016
:100220004F004D001F001A0015001B0001582A0046
:100230002000090016000600E300286821001300D2
:1002400017001900E2004A0022000A00070005001A
:10025000000049002A002F000000D45C0000035871
:100260002E0030000000D55C0000330223000D009A
:100270000B000E000000007424000F00110010009D
:1002800000674B002500180008003600E4002C62CF
:1002900026001C000C00370002584C0027003300D9
:1002A0001200380051004E002D0031003472E4007D
:1002B00052000000290001000100010001000000BF
:1002C0003A001E0220022202010001003B001F0230
:1002D00021022302010001003C002F0226022F0010
:1002E000010001003D003002270230000100010042
:1002F0003E0031023500350200000100010001001E
:1003000000000100000001000100010000000100E8
:10031000000001003F0052005100240200000100D3
:100320004000240021001E000100010041002500C2
:1003300022001F0037000100420026002300200099
:1003400027000100430025022E0231002E0001008B
:10035000440045000100010001000000010001000F
:100360000100010001000000010001000100010086
:100370000100010001000100F200FB00F900F5009E
:100380000100F000F1000100F600F400010001009E
:10039000F300FC00FA00010001000100010001006F
:1003A0000000010001000100000001000000010048
:1003B0000100010000000100000001000100010037
:1003C0000B00010000000100010001000D00010010
:1003D00001000100010001000E0001000100010008
:1003E000010001000F0001000100010001000100F7
:1003F00033000100010001000100010001000100C3
:10040000010000000C000F000000000000000000D0
:1004100029002B002B00E100000001001E00140049
:1004200004001D00000001001F001A0016001B0040
:10043000E0002C002000080007000600E200010098
:1004400021001500090019000000010022002E0003
:100450000000100000000100010001000000010088
:100460000000010001003A0001000100000001004D
:1004700001003B00010001000100010001003C00FF
:10048000010001000100010001003D000100010028
:100490000100010001003E00010001000100010017
:1004A0000100010001000100010000000000000047
:1004B000000000002A2B28000000000000000000BF
:1004C0000000000000000029000000002C1E342065
:1004D000212224342627252E362D3738271E1F208B
:1004E0002122232425263333362E37381F040506D0
:1004F0000708090A0B0C0D0E0F1011121314151614
:100500001718191A1B1C1D2F3130232D3504050611
:100510000708090A0B0C0D0E0F10111213141516F3
:100520001718191A1B1C1D2F3130354C0000000004
:1005300000000000000000000000000000000000BB
:1005400000000000000000000000000000010101A8
:100550000101010001010101000000000000000094
:100560000000000000000100010001010101010183
:10057000010101010101010101010101010101016B
:100580000101010101010100000001010000000062
:10059000000000000000000000000000000000005B
:1005A0000000000000000001010101006801F000EE
:1005B000B40078005A007F3F1F643214643214780C
:1005C0003C1E1E140A05000000000001010101018B
:1005D00001010101020202020202020202030303FC
:1005E00003030303030404040404040505050505CB
:1005F0000606060606070707070808080809090986
:100600000A0A0A0A0B0B0B0C0C0C0D0D0D0E0E0F2B
:100610000F0F1010111111121213131414151516B7
:10062000161717181819191A1A1B1C1C1D1D1E1F26
:100630001F20202122222324252526272728292A76
:100640002B2B2C2D2E2F2F3031323334353636379D
:1006500038393A3B3C3D3E3F40414243444647489F
:10066000494A4B4C4D4F50515253555657585A5B6F
:100670005C5E5F606263646667696A6C6D6E707110
:1006800073747678797B7C7E8081838486888A8B7C
:100690008D8F91929496989A9B9D9FA1A3A5A7A9AF
:1006A000ABADAFB1B3B5B7B9BBBDBFC1C4C6C8CAA6
:1006B000CCCFD1D3D6D8DADCDFE1E4E6E8EBEDF05D
:1006C000F2F5F7FAFCFF16034500720067006F00B1
:1006D00044006F007800200045005A000000160317
:1006E0004500720067006F0044006F007800200032
:1006F00045005A0000000403090409026D000401CA
:1007000000A0FA0904000001030101000921110100
:1007100000012240000705810308000A09040100C6
:100720000103010200092111010001224D0007050A
:10073000820308000A0904020001030000000921E5
:10074000110100012236000705830308000A09048D
:1007500003000103000000092111010001223900FA
:10076000070584032000011201100100000008EDBC
:10077000FE071301000102000105010906A10105A0
:100780000719E029E7150025019508750181020583
:1007900008190129059505750191029501750391C7
:1007A000010507190029F71500250195F875018144
:1007B00002C005010980A10185021601002603007F
:1007C0001A81002A8300751095018100C0050C096B
:1007D00001A1018503160100269C021A01002A9C32
:1007E00002751095018100C005010902A1010901EE
:1007F000A1000509190129051500250195057501B7
:1008000081029501750381010501093009311581C6
:10081000257F95027508810609381581257F950188
:1008200075088106050C0A38021581257F9501752A
:10083000088106C0C005010906A101050719E029C4
:10084000E71500250195087501810295017508815C
:100850000105081901290595057501910295017594
:100860000391010507190029FF150026FF009506D1
:1008700075088100C00011241FBECFEFDAE0DEBF93
:10088000CDBF04B603FE27C08091BA039091BB038D
:10089000A091BC03B091BD038730904BA740B04BF3
:1008A000D1F41092BA031092BB031092BC031092C1
:1008B000BD0314BE84B7877F84BF0FB6F894A89594
:1008C00080916000886180936000109260000FBE8C
:1008D000E0E0FFE3099511E0A0E0B1E0E2EEF3E62D
:1008E00002C005900D92AC3DB107D9F723E0ACED05
:1008F000B1E001C01D92AA3BB207E1F70E94D128E6
:100900000C94EF310C9400001092B9008AE08093AF
:10091000B800089594EA9093BC009091BC0097FFB2
:10092000FCCF9091B900987F983021F0903111F070
:1009300081E008958093BB0084E88093BC0080919F
:10094000BC0087FFFCCF8091B900887F883111F00F
:10095000803471F780E0089584E98093BC00809131
:10096000BC0084FDFCCF08958093BB0084E8809395
:10097000BC008091BC0087FFFCCF9091B900987FAC
:1009800081E0983209F480E0089584E88093BC0007
:100990008091BC0087FFFCCF8091BB00089580B39D
:1009A0008C7080BB81B3836F81BB089580910001FF
:1009B000811115C080E40E948A0480930001811196
:1009C0000CC082E10E94B40480930001811105C033
:1009D0008FEF0E94B404809300010E94AC0484B1A4
:1009E000807F84B985B1807F85B98AB1837F8AB9D8
:1009F0008BB1837F8BB93E984698089508950C94E7
:100A0000FE040E94C406809300010E94D6040E9446
:100A1000CF042DED31E0E1E3F2E04EE04E0F119214
:100A200080E090E0D901A80FB91F1C920196863092
:100A30009105C1F72A5F3F4F4E13F1CF0C947A0A0C
:100A40000E94C406809300010E94D6040E94CF0435
:100A5000E1E3F2E08EE08E0F11928E13FDCF089548
:100A600026E0829FC0011124FC01E352FE4F20E0EA
:100A700030E080E041E050E09081992319F09150FE
:100A8000908307C0BA01022E01C0660F0A94EAF7EC
:100A9000862B2F5F3F4F31962630310569F7089539
:100AA00096E0699FB001112420E030E090E04FE033
:100AB000FC01022E02C0F595E7950A94E2F7E0FFEB
:100AC00006C0F901E60FF71FE352FE4F40832F5F88
:100AD0003F4F2630310561F70895AF92BF92CF9214
:100AE000DF92EF92FF920F931F93CF93DF9380914A
:100AF0000001882379F08091DC018F5F8093DC0115
:100B0000811108C00E94C40680930001811102C0B7
:100B10000E94560681E3E82E82E0F82E00E010E005
:100B2000CC24C394D12CAA24A394C02F0730110540
:100B300000F58091000181113CC080E40E948A048C
:100B400080930001811112C082E10E94B40480935D
:100B5000000181110BC0C601002E01C0880F0A944C
:100B6000EAF780950E94B404809300010E94AC04CF
:100B700020C00A30A1F028F4083059F0093061F0A3
:100B800005C00C3089F070F00D3089F0209A28985B
:100B900010C0219A29980DC0229A2A980AC0239A37
:100BA0002B9807C0529A01C0539A5B9802C03E9A94
:100BB000469880EA8A95F1F78C2F0E943005D82F4D
:100BC0000730110518F580910001811144C080E4BF
:100BD0000E948A0480930001882311F0B12C12C076
:100BE00083E10E94B404809300018111F7CF81E476
:100BF0000E948A04809300018111F0CF0E94C504F5
:100C0000B82EB0940E94AC049B2D26C08FB1817089
:100C10008A25799902C092E001C090E0892B7C99E5
:100C200002C094E001C090E0982B7D9902C038E0AA
:100C300001C030E0932B7E9902C020E101C020E08A
:100C4000922B2FB12095221F2227221F2295220F9F
:100C5000207E922B01C090E0F70180819D23D095EA
:100C6000D823D92B6C2F8D270E945005F701D193E3
:100C70007F010E94D6040F5F1F4F0E30110509F04F
:100C800054CF0E947C0A81E0DF91CF911F910F9198
:100C9000FF90EF90DF90CF90BF90AF900895E82F36
:100CA000F0E0EF5CFD4F80810895089556985E98BE
:100CB00025982D9826982E9827982F988FEF90E0BA
:100CC000909389008093880090938B0080938A0092
:100CD00090938D0080938C00259A2D9A2FEF80E7BA
:100CE00092E0215080409040E1F700C00000269A39
:100CF0002E9A2FEF80E792E0215080409040E1F75C
:100D000000C00000279A2F9A2FEF80E792E0215031
:100D100080409040E1F700C0000025982D982FEF0B
:100D200080E792E0215080409040E1F700C0000051
:100D300026982E982FEF80E792E021508040904037
:100D4000E1F700C0000027982F9856985E982598E4
:100D50002D9826982E9827982F98089589EA8093A1
:100D6000800089E08093810024982C983F988AB174
:100D70008F7C8AB96E98479A8BB180638BB9769ACB
:100D80000E9456060C94200780E280930001809117
:100D90003F0281110EC00E94840481E080933F02D3
:100DA0002FEF83ED90E3215080409040E1F700C0A9
:100DB000000080E40E948A048093000181112EC00B
:100DC0000E94B40480930001811128C00E94B404E1
:100DD00080930001811122C08FE30E94B4048093AC
:100DE000000181111BC00E94AC0480E40E948A04AF
:100DF00080930001811112C08CE00E94B4048093A2
:100E0000000181110BC00E94B40480930001811184
:100E100005C08FE30E94B404809300010E94AC04DB
:100E2000809100010895611108C0FC01828188232E
:100E300021F083ED91E00E94770A80E090E0089530
:100E40000895FB018C3D2CE5920769F08D3D2CE562
:100E5000920789F08B3D9C45B1F482818823A1F0F3
:100E60000E9401210EC08281882371F08EE991E0F9
:100E70000E94770A06C08281882331F081E00E94B7
:100E8000A01080E0089581E00895CF92DF92EF9264
:100E9000FF926B017C010E94B12056985E982598C4
:100EA0002D9826982E9827982F9890E0FC0131973E
:100EB000E730F105A8F4EA5AFF4F0C94A131259AC6
:100EC0002D9A0EC0259A2D9A269A2E9A09C0259AF7
:100ED0002D9A04C0259A2D9A269A2E9A279A2F9AEF
:100EE000C701B601FF90EF90DF90CF90089581E0A9
:100EF00008950C9421070E94851A2FEF84E39CE04B
:100F0000215080409040E1F700C000000C948D22F9
:100F1000FF920F931F93CF93DF938C01FC01C0814D
:100F2000D18180919102811113C08281882349F07F
:100F3000CE010E94A71FF82E682FCE010E944A1FE3
:100F400004C0CE010E947A1FF82EBE018F2D04C06E
:100F5000CE010E94A71FBE010E94910AEC01B801B8
:100F60000E947907882309F462C2B801CE010E9469
:100F7000ED0C882309F45BC2B801CE010E943C0D40
:100F8000882309F454C2CA3CFCE5DF0741F4F801A8
:100F90008281882309F44BC20E946B1048C2CB3C6B
:100FA0008CE5D80708F004C1C33C9CE5D90741F49F
:100FB000F8018281882309F43AC20E942E1137C2B7
:100FC000C43CECE5DE0708F0ACC0C531FCE5DF074A
:100FD00008F057C0C2308CE5D80708F47BC0F80190
:100FE0008281882309F46EC00E942221811102C0EF
:100FF0000E9401210E94352190E09093AC038093E0
:10100000AB03FE01E350FC45E231F10530F4E35A55
:10101000FF4F8091AB030C94A1318091AB038160B1
:1010200027C0826025C0846023C0806121C08062A7
:101030001FC080641DC080681BC08460886018C0A9
:101040008E7F16C08D7F14C08B7F12C08F7E10C024
:101050008F7D0EC08F7B0CC08F770AC08B7F877F00
:1010600007C087FB222720F991E0922790FB87F9A0
:101070008093AB038091AB030E9439210E94851AB3
:10108000D6C1C531DC45C9F40E947820282FF8016B
:10109000828140910301509104018823B9F12A7A99
:1010A00091E009F490E09093400291112DC069E223
:1010B000CA010E949A210E94452081E08093450246
:1010C00080934602C801DF91CF911F910F91FF904D
:1010D0000C947707C1159CE5D90741F4F80182818A
:1010E000882309F4A4C10E947B07A1C1C130DC455B
:1010F00021F7F8018281882309F499C180912F0397
:10110000816080932F0393C165E3D2CF8091400229
:10111000811102C069E201C065E3CA010E94A521F4
:10112000CACFC63C8CE5D80741F4F80182818823F8
:1011300009F47DC10E9410107AC1C73C9CE5D90713
:10114000E0F4C43CECE5DE0741F4F8018281882339
:1011500009F46DC10E941B116AC1C53CDC4509F050
:10116000ACCFF8018281882309F461C10E94782004
:10117000827281F30E9425115AC1F8018281C83C14
:10118000FCE5DF0731F4882309F451C10E944710C0
:101190004EC1C93CDC4530F4882309F448C10E94A3
:1011A000281045C1882309F442C10E9459103FC14B
:1011B000C13DECE5DE07C1F4F8018281882309F422
:1011C00036C10E94E60E653171058105910540F03A
:1011D0000E94E60E673171058105910508F4BACFCA
:1011E00085E10E94A01023C1C23DFCE5DF0708F0A5
:1011F0007AC0CD3C8CE5D807B1F4F8018281882310
:1012000009F415C10E94E60E623071058105910551
:1012100040F00E94E60E653071058105910508F4E5
:1012200099CF82E0DECFCE3C9CE5D907B8F4CB3C29
:10123000ECE5DE0741F4F8018281882309F4F7C068
:101240000E948610F4C0CC3CDC4509F036CFF80192
:101250008281882309F4EBC081E0C3CFF801828149
:10126000CF3CFCE5DF07A1F4882309F4E0C00E942D
:10127000E60E693071058105910540F00E94E60E89
:101280006E3071058105910508F464CF89E0A9CF1E
:10129000C03DDC45A0F4882309F4C9C00E94E60ED5
:1012A000663071058105910540F00E94E60E6830B8
:1012B00071058105910508F44DCF86E092CF882312
:1012C00009F4B5C00E94E60E6F30710581059105E5
:1012D00040F00E94E60E643171058105910508F425
:1012E00039CF8FE07ECFC43DECE5DE0761F5F80134
:1012F0008281882351F0109245020E9431229093FE
:1013000042028093410282E03DC00E94782085FF26
:1013100005C081E08093450280934602809145029A
:1013200081110FC080914102909142020E943D22A2
:10133000883C910530F486E20E94171686E20E94EE
:10134000261782E030C0C53DFCE5DF0778F1C83DD7
:10135000ECE5DE0709F44DC0C93DFCE5DF0709F403
:101360004EC0C53DDC4509F0A8CEF8018281882336
:1013700061F0109246020E943122909344028093C1
:10138000430280E20E94851752C00E94782081FFAC
:1013900005C081E080934502809346028091460219
:1013A0008823A9F180E20E948C1741C0C23D8CE5E0
:1013B000D80731F4F80182818823C9F188E111CF7F
:1013C000C33DDC4509F079CEF8018281882379F1AB
:1013D0000E94E60E693171058105910540F00E9479
:1013E000E60E623271058105910508F4B3CE89E1FC
:1013F000F8CEF80182818823D1F080E005C0F801A1
:1014000082818823A1F082E00E94672910C0809128
:101410004302909144020E943D22883C910510F6BF
:1014200087E20E94171687E20E942617BBCF80E052
:10143000DF91CF911F910F91FF900895CF93282FA7
:1014400030E0F901E455FB4FC491F901E45DFA4F36
:101450002491222359F081EE0E9417168C2F0E94AE
:1014600017168C2F0E94261781EE04C08C2F0E9425
:1014700017168C2FCF910C9426170F931F93CF9391
:10148000DF93EC01062FFE018491882359F19E0120
:101490002F5F3F4F813041F4E901F9011491812F11
:1014A0000E941716812F0DC0823031F4E901F90135
:1014B00084910E9417160AC0833031F4E901F901C2
:1014C00084910E94261702C00E941E0A2196802F36
:1014D0008823C9F2EFE9FFE03197F1F700C000007F
:1014E0008150F6CFDF91CF911F910F91089560E069
:1014F0000C943D0A0C94AE060C94FF04282F88230C
:1015000039F090E02A3010F44D960895069708952A
:1015100087E290E0089508950C948B0A0C948C0A4D
:10152000089596E0799FF001112494E5899FE00DDC
:10153000F11D1124E60FF11DEE0FFF1FE45FFD4FBB
:10154000859194910895880F991FFC01E85FFD4FE4
:10155000859194910895CF93DF930E94910A0E9400
:10156000430CEC01811520E49207B0F5811540E3AE
:10157000940708F0E1C0803E9105D0F4803C9105CD
:1015800008F06FC0883A910570F4853A910508F02B
:101590006BC08130910509F472C108F429C1049728
:1015A00008F06DC125C18D3B910508F468C020C1CC
:1015B0008F3F910509F048F4803F910508F0B6C0CF
:1015C000883E910508F45BC113C1811550E295076F
:1015D00008F455C19F70ACC0811564E59607D8F436
:1015E000C11583E5D80708F0E2C0C11521E5D2078F
:1015F00040F4C11540E5D40708F0A7C0DF70D06AF9
:101600003EC1C11552E5D50708F0BBC0DC2FCC2781
:10161000C16FD06A34C1811566E5960750F4C115D3
:1016200085E5D80708F0D9C0DC2FCC27C46FD06A75
:1016300026C1811528E5920708F4DAC0811549E52D
:10164000940708F4D0C090568115904208F0D0C09D
:101650008D2F8F710E94C00CDD27D0628F71D82B27
:101660000EC1805C910964C0853A910509F4C3C03C
:10167000863A910509F0C2C0C2E8D0E400C1883AB8
:10168000910509F4BEC0893A910509F4BDC08A3AB2
:10169000910509F4BCC08B3A910509F4BBC08C3AA2
:1016A000910509F4BAC08B3B910509F4B9C08C3B94
:1016B000910509F4B8C08D3A910509F4B7C0803B93
:1016C000910509F4B6C08E3A910509F4B5C08F3A78
:1016D000910509F4B4C0813B910509F4B3C0823B84
:1016E000910509F4B2C0833B910509F4B1C0843B74
:1016F000910509F4B0C0853B910509F4AFC0863B64
:10170000910509F4AEC0873B910509F4ADC0883B53
:10171000910509F4ACC0893B910509F4ABC08A3B43
:10172000910509F4AAC0C0E0D4E4A9C0D065A7C05F
:101730000E94A30AEC01A3C09927D3FF03C0EC01C8
:10174000D86C9DC0EC01D06C9AC02C2F237081E026
:1017500090E002C0880F991F2A95E2F79C689E01CD
:1017600044E0369527954A95E1F72370922BCF7088
:10177000C695C69560E2C69FE0011124C82BD92BFF
:101780007EC02C2F2695269580E2289F900111245B
:10179000C370DD2781E090E0AC0102C0440F551F0B
:1017A000CA95E2F7EA01C22BD32BDC6868C02C2F64
:1017B0002695269580E2289F90011124C370DD278D
:1017C00081E090E0AC0102C0440F551FCA95E2F7DA
:1017D000EA01C22BD32BDA6852C0CF71DD27DC2F90
:1017E000CC27D0624CC0DC2FCC27C06FD06A47C05A
:1017F000C0E0D0E044C0C1E8D0E441C0C3E8D0E4D8
:101800003EC0C2EED4E43BC0C9EED4E438C0CAEE58
:10181000D4E435C0C5EBD4E432C0C6EBD4E42FC069
:10182000C3EBD4E42CC0C4EBD4E429C0C7EBD4E4AC
:1018300026C0CCECD4E423C0CDECD4E420C0C3E873
:10184000D5E41DC0CAE8D5E41AC0C2E9D5E417C082
:10185000C4E9D5E414C0C1E2D6E411C0C3E2D6E4C1
:101860000EC0C4E2D6E40BC0C5E2D6E408C0C6E2AE
:10187000D6E405C0C7E2D6E402C0CAE2D6E4CE018F
:10188000DF91CF9108958238910549F1B0F4813309
:10189000910509F458C048F48932910509F44EC005
:1018A0008A32910509F454C008958533910509F4ED
:1018B00040C08933910599F00895833E910529F13F
:1018C00038F4803E910591F0823E9105A1F0089593
:1018D000863E9105F9F0873E910531F108952091FA
:1018E000AB0320FD3AC021FD38C008958091AB03C1
:1018F00080FD35C032C08091AB0382FF32C0809141
:10190000AB0384FD30C083EE39C08091AB0382FD10
:1019100028C0F5CF8091AB0383FF27C08091AB0334
:1019200084FD21C087EE2AC08091AB0383FD1DC0DA
:10193000F5CF8091AB0385FD1AC01BC08091AB032E
:1019400085FD17C014C08091AB0386FD14C015C07F
:101950008091AB0386FD11C00EC080EE0FC089E3FD
:101960000DC082EE0BC080E009C086EE07C089E2A0
:1019700005C085E303C08AE201C081E390E00895D9
:10198000CF93C82F0E94352190E09093AC038093B1
:10199000AB0382FF0DC09C2F9871983019F4C77F5C
:1019A000C46006C09C2F9471943011F4CB7FC86042
:1019B00083FF0DC09C2F9871983119F4C77EC461C4
:1019C00006C09C2F9471943111F4CB7EC86184FDC4
:1019D000C77E8C2FCF91089508950F931F93CF93B7
:1019E000FB012281211102C0C1E041C08C01C091E4
:1019F0005402C11125C086319C45B1F70E94EC0C00
:101A000081E0809354020E9431229093530280938C
:101A1000520210924702109249021092480210920C
:101A20004B0210924A0210924D0210924C021092F8
:101A30004F0210924E02109251021092500217C0A3
:101A400080915202909153020E943D22883C910560
:101A500058F690914702E92FF0E0EE0FFF1FE85B88
:101A6000FD4F118300839F5F90934702C0E08C2F4E
:101A7000CF911F910F910895CF93DF93813020E88C
:101A80009207D0F0FB0122812223B1F0EC0180917A
:101A90005502811109C08CE090E00E94A7310E949C
:101AA000600D81E0809355020E94670DCE019F7703
:101AB0000E942F0E0E94E30D81E0DF91CF910895E7
:101AC00080935602682F8CE090E00C94BB31E0913B
:101AD0000301F091040180818093600381FF03C0C2
:101AE00081EE0E9426178091600385FF03C085EE7A
:101AF0000E9426178091600380FF03C080EE0E9441
:101B000026178091600384FF03C084EE0E9426178D
:101B10008091600382FF03C082EE0E9426178091AD
:101B2000600386FF03C086EE0E9426178091600343
:101B300083FF03C083EE0E9426178091600387FF16
:101B400003C087EE0E94261780915602823001F171
:101B5000A8F48823C9F0813079F580EE0E94171629
:101B600081EE0E94171688E10E94171688E10E94F4
:101B7000261781EE0E94261780EE1CC0843081F06B
:101B80008530D1F486EE01C082EE0E94171614C093
:101B900082EE0E94171687E50E94171687E50AC095
:101BA00086EE0E94171686EE0E94261788E10E9494
:101BB000171688E10E9426178FE39CE90197F1F739
:101BC00000C00000089580915602813049F030F045
:101BD000823021F0853051F486EE06C082EE04C0DA
:101BE0008CE20E9417168CE20E94261780916003F7
:101BF00081FF03C081EE0E9417168091600385FF6C
:101C000003C085EE0E9417168091600380FF03C019
:101C100080EE0E9417168091600384FF03C084EE5B
:101C20000E9417168091600382FF03C082EE0E941B
:101C300017168091600386FF03C086EE0E94171678
:101C40008091600383FF03C083EE0E94171680918A
:101C5000600387FF03C087EE0C9417160895EF9278
:101C6000FF921F93CF93DF937C01CCE0D0E09701EC
:101C70000C2E02C0369527950A94E2F7122F1F709A
:101C8000812F0E947E0A0E941716812F0E947E0AD1
:101C90000E9426172497CC3F8FEFD80741F7DF919A
:101CA000CF911F91FF90EF900895EF92FF920F93C5
:101CB0001F93CF93DF93E901662309F44BC0242FD0
:101CC00030E0EFEFF0E0E61BF109B901E69F90018B
:101CD000E79F300DF69F300D1124232F8B01031B3E
:101CE00011095CE3E52EF12CB7010E947931FB016B
:101CF000BC01069FC001079F900D169F900D1124F7
:101D0000B7010E947931E230F105B1F040F430972B
:101D100079F0319711F5832F242F461B21C0E43031
:101D2000F105A1F068F03597C1F4842F861B18C027
:101D3000832F262F230F14C0862F830FE42F03C079
:101D4000E42FE61B842F432F2E2F0AC0842F462F0B
:101D5000430F06C0842F242F03C080E020E040E022
:101D6000E42FF0E0EA53FA4F4491E22FF0E0EA5317
:101D7000FA4F9491E82FF0E0EA53FA4FE491498347
:101D80009883EA83DF91CF911F910F91FF90EF909D
:101D9000089588E090E00C94AF31AB01BC0188E07D
:101DA00090E00C94CD31E1E6F3E083E08083109283
:101DB00062038FEF8283838360916103709162037A
:101DC00080916303909164030C94CD0E6091610344
:101DD00060FF06C066956F7370E080E090E0089544
:101DE00060E070E0CB0108958091610380FF06C040
:101DF0006FE070E089E693E00C94541480E090E08A
:101E0000FC01E759FC4F11821082128204968C3338
:101E10009105B1F7EDCF20E030E0F901E759FC4F33
:101E20008183608342832C5F3F4F2C333105A9F7B8
:101E30000C94F40EEF92FF920F931F93CF93DF93C6
:101E400000D000D0CDB7DEB70091610310916203DE
:101E5000209163033091640300936503109366033C
:101E600020936703309368032091610320FF21C012
:101E7000042FF62EE92E182F9E012F5F3F4F0E9450
:101E8000550E8091650310FB87F9809365031695C5
:101E9000809166038078182BE0FA17F91093660397
:101EA000F0926703009368034B8169818A810E94E5
:101EB0000B0F0F900F900F900F90DF91CF911F910C
:101EC0000F91FF90EF9008958F929F92AF92BF92E3
:101ED000CF92DF92EF92FF920F931F93CF93DF93F6
:101EE000EC01062F142F8091610380FF8CC0982F86
:101EF0009E77923021F4CE010E941A0F5AC0E82F2B
:101F0000E695EF739EE39E0F9F73943018F4109143
:101F100064034FC09AE39E0F9F73993070F4881F3B
:101F20008827881F90916203292F220FC22FC82B68
:101F300097FB992790F9D92F3CC087E28E0F8F73BA
:101F40008A30B8F5F0E07997E0FD02C021E001C0E9
:101F50002FEFEE7FE455FA4F859194916FE070E09A
:101F60000E94793126036001279FD00C11244E0175
:101F700088E9881A8EEF980A89E6E82E83E0F82E21
:101F800098E6A92EBB24B394C401B5010E9479310F
:101F90009701412F602F0E94550E8C0C9D1C94E0E0
:101FA000E90EF11C85EAE81683E0F80669F70E945D
:101FB000F40E809161039C2FC0FB87F9809361032D
:101FC0009695809162038078892BD0FB87F9809366
:101FD0006203009363031093640360916103709143
:101FE00062038091630390916403DF91CF911F910D
:101FF0000F91FF90EF90DF90CF90BF90AF909F90A8
:102000008F900C94CD0EDF91CF911F910F91FF9087
:10201000EF90DF90CF90BF90AF909F908F900895FA
:10202000E1E6F3E02081221F2227221F3091620384
:10203000432F440F842F822B37FB992790F90C965E
:1020400068E671E00E948D31438162810C94640FD7
:1020500020916103221F2227221F30916203432F08
:10206000440F842F822B37FB992790F98C309105F0
:102070001CF4845A9E4F01C00C9768E671E00E94E0
:102080008D3140916403609163030C94640FE1E629
:10209000F3E08081881F8827881F90916203292F91
:1020A000220F97FB992790F943816FEF822B0C94B5
:1020B000640FE1E6F3E08081881F8827881F9091F4
:1020C0006203292F220F97FB992790F9438160E043
:1020D000822B0C94640F40916403842F90E0843F22
:1020E000910514F4445F01C04FEF80916103881F94
:1020F0008827881F90916203292F220F97FB992729
:1021000090F960916303822B0C94640F40916403F7
:10211000842F90E00C9714F04C5001C040E0809167
:102120006103881F8827881F90916203292F220F3F
:1021300097FB992790F960916303822B0C94640FAD
:102140009091610390FF42C09178811102C092602A
:1021500007C0833210F0946403C08F73880F982BEC
:1021600090936103609161037091620380916303B6
:10217000909164030E94CD0E80916103982F9E7709
:10218000923019F410926C0210C0982F96959F739C
:102190002EE3290F2F73273120F491E090936C02E6
:1021A00004C0995D9F739A3068F3881F8827881F41
:1021B00090916203292F220F97FB992790F9409164
:1021C000640360916303822B0C94640F08958091E3
:1021D0002F03816080932F0381E080936D020E9422
:1021E0002221811104C00E9401210E94D30E0E946D
:1021F000C90E6093610370936203809363039093AD
:1022000064036E7761F40E94D30E0E94C90E60933E
:10221000610370936203809363039093640381E08E
:1022200080936C028091610380FF04C086958F7358
:102230000C94A01008958091610386958F738F5F31
:10224000833208F081E00C94A010809161038695A0
:102250008F73815009F482E20C94A0108091610385
:10226000982F909590FB80F98093610360916103B2
:102270007091620380916303909164030E94CD0E7C
:102280008091610380FF04C086958F730C94A01029
:1022900010926C022FEF80E792E021508040904036
:1022A000E1F700C000000C94F40ECF93C82F80918A
:1022B0006A0290916B020E943D22EC2FF0E0EE53F7
:1022C000FA4FE491F0E08E179F0708F443C00E9494
:1022D000312290936B0280936A026091690270E0F0
:1022E00080E090E00E947A2F20E030E04FE753E456
:1022F0000E949D2E2BED3FE049E450E40E94A33064
:102300000E9410310E94172F2BE43AE34EE25FE364
:102310000E94302E20EF3BEF48ED52E40E94A330A4
:102320000E94492F462F80916103881F8827881FAC
:1023300090916203292F220F97FB992790F96091C2
:102340006303822B0E941A0F8091690290E001962C
:1023500080936902CF910895CF93C82F809167022F
:10236000909168020E943D22EC2FF0E0E154FA4F78
:10237000E491F0E08E179F07E8F00E9431229093DD
:1023800068028093670240916403609163038091C7
:102390006502909166020E941A0F809165029091E9
:1023A0006602019668E671E00E94793190936602B8
:1023B00080936502CF910895CF92DF92FF920F93A1
:1023C0001F93CF93DF93F82E809163029091640264
:1023D0000E943D22EF2DE695F0E0E454FA4FE4919F
:1023E000F0E08E179F07E8F10E943122909364027B
:1023F0008093630209E613E0C0E0D0E088E6C82ECF
:10240000DD24D39480916102909162028C0F9D1F14
:10241000B6010E9479319801409164036091630391
:102420000E94550E68960C5F1F4FC83681E0D80792
:1024300049F70E94F40E2091610230916202F0FE91
:102440000AC0C9010196BE010E94793190936202CF
:102450008093610206C021503109309362022093BB
:102460006102DF91CF911F910F91FF90DF90CF908C
:102470000895AF92BF92CF92DF92EF92FF920F93A7
:102480001F93CF93DF93C82F80FF02C01FEF01C0BF
:1024900011E080915F02909160020E943D22C695FA
:1024A000EC2FF0E0E754FA4FE491F0E08E179F072D
:1024B00008F466C00E9431229093600280935F020C
:1024C00029E6C22E23E0D22E3BE6E32E33E0F32EA4
:1024D000C0E0D0E0F70131971082F6011082F701D9
:1024E000108294E0A92EB12C00E080915E02800F52
:1024F00087FD815F082E000C990BC817D907E9F4F6
:10250000809164038A9DA0018B9D500D11245595E7
:1025100047955595479580916103881F8827881FA7
:1025200090916203592F550F97FB992790F99601C7
:1025300060916303852B0E94550E010FF1E0AF1AE5
:10254000B10899F6219684E0C80ED11CE4E0EE0EA5
:10255000F11CCF30D10509F0BDCF0E94F40E80915F
:102560005E02113031F4811102C08EE007C081504B
:1025700005C090E00196BE010E948D3180935E02FD
:10258000DF91CF911F910F91FF90EF90DF90CF904F
:10259000BF90AF9008950F931F93CF93DF93C82FF1
:1025A00080915C0290915D020E943D22EC2FF0E050
:1025B000EA54FA4FE491F0E08E179F0708F464C0E4
:1025C0000E94312290935D0280935C0280E090E053
:1025D000FC01E759FC4F11821082128204968C3361
:1025E0009105B1F7C0E0D0E00FE010E0CE01B801F6
:1025F0000E948D31FC0180915B02082E000C990B2A
:10260000EE0FFF1FEE0FFF1FC817D907FCF08091D8
:102610000201082E000C990B8C179D07BCF09F013E
:1026200027593C4F80916103881F8827881F90910C
:102630006203592F550F97FB992790F94091640336
:1026400060916303852B0E94550E05C0E759FC4F2E
:102650001182108212822196CF30D10539F60E9464
:10266000F40E8091010190915B02980F90935B02B0
:1026700020910201280F20930201121614F49E30BB
:102680001CF0819580930101DF91CF911F910F91F3
:102690000895EF92FF920F931F93CF93DF93809152
:1026A000590290915A020E943D22883E9340D0F1F7
:1026B0000E94312290935A0280935902C09157028E
:1026C000D09158022196C170DD27D0935802C09353
:1026D000570289E6E82E83E0F82E10E008E7812F04
:1026E0008695FE01E80FF11DCF01817099279701B2
:1026F0004091640360916303FC010E9FC0010F9F32
:10270000900D11240E94550E1F5FF4E0EF0EF11C96
:102710001F3029F7DF91CF911F910F91FF90EF901C
:102720000C94F40EDF91CF911F910F91FF90EF90D9
:10273000089580916C02882391F190916103892F13
:1027400086958F732EE3280F2F73243018F4825050
:102750000C9455112AE3280F2F73233018F4865058
:102760000C94AC1127E3280F2F73263018F48950EE
:102770000C94DC1121E3280F2F73263018F48F50AE
:102780000C9439122BE2280F2F73233018F4855143
:102790000C94CB129E77903311F40C944913089546
:1027A000882319F05198599A02C0519A5998509813
:1027B000589A95E09A95F1F70000509A589895E04C
:1027C0009A95F1F70000882311F0519A599885E005
:1027D0008A95F1F7000008958BB18C7F8BB95098E2
:1027E000589A5198599A85E08A95F1F70000089512
:1027F0008AB18C7F8AB985E08A95F1F70000519AF9
:10280000599885E08A95F1F70000509A589885E02C
:102810008A95F1F7000008955098589A85E08A95B6
:10282000F1F700005198599A85E08A95F1F7000078
:102830000895CF93DF93D82FC8E08D2F80780E9422
:10284000D013DD0FC150C9F780E00E94D01385E09E
:102850008A95F1F7000085E08A95F1F7000080E0A5
:10286000DF91CF9108952BB1342F309523233BB1C5
:10287000432B3FB7F894FC01680F791FE617F70761
:1028800089F0819198E04BB9000000C087FF2BB917
:10289000880F000000C000C000C02BB900C09A958E
:1028A00091F7ECCF3FBF0895AF92BF92CF92DF92E6
:1028B000EF92FF920F931F93CF93DF938C01EB0165
:1028C000CFB6D090BC00F8948091BC008B7F8093F1
:1028D000BC000E94EC130E94F81384E80E941914B3
:1028E000CC0FDD1FCC0FDD1F78015801AC0EBD1ED3
:1028F000EA14FB0431F0F70181917F010E94191461
:10290000F7CF0E940C14CFBED092BC00579A40E87B
:10291000BE01C801DF91CF911F910F91FF90EF9001
:10292000DF90CF90BF90AF900C94331490937302CC
:10293000809372020895E0917202F09173023097D1
:1029400021F00190F081E02D099480E00895E0915C
:102950007202F0917302309721F00280F381E02D32
:1029600009940895E0917202F0917302309721F07A
:102970000480F581E02D0994089520917002309132
:1029800071028217930771F0909371028093700225
:10299000E0917202F0917302309721F00680F78186
:1029A000E02D0994089520916E0230916F028217F4
:1029B000930771F090936F0280936E02E091720220
:1029C000F0917302309721F00084F185E02D099495
:1029D000089508950C94E91481E008950E94282236
:1029E0000E9401050E94AF220C94E710CF92DF9263
:1029F000EF92FF920F931F93CF93DF93CDB7DEB784
:102A00002B970FB6F894DEBF0FBECDBF0E946D05A9
:102A10000E94EC14811111C08FEF89838A831B827D
:102A20000E9431228160782F9D838C8349815A8155
:102A30006B818D810E94DA1556C085E7C82E82E031
:102A4000D82E00E010E0E02E802F0E944F06F60105
:102A500041916F01F42EF82631F40F5F1F4F0E30B5
:102A6000110589F7D9CF90912F0391FF04C08B876F
:102A70000E9455068B8520E030E04F2D50E0922FCC
:102A8000BA01022E02C0759567950A94E2F760FFBD
:102A900024C02E83EF8221E030E0690102C0CC0C1B
:102AA000DD1C9A95E2F790E08C219D21892B09F499
:102AB00020E028870E9431228160782F9A878987B9
:102AC0004E815F8168858A850E94DA15F801EB588E
:102AD000FD4F8081C826C08206C02F5F3F4F263041
:102AE000310569F6BACF0E944224109174020E9407
:102AF0009B141817A1F00E949B14809374022B96CC
:102B00000FB6F894DEBF0FBECDBFDF91CF911F91FE
:102B10000F91FF90EF90DF90CF900C948E0A2B9640
:102B20000FB6F894DEBF0FBECDBFDF91CF911F91DE
:102B30000F91FF90EF90DF90CF900895DC011196F8
:102B40002C9111978C91682F70E041E050E001C00A
:102B5000440F8A95EAF712968C91129730E08823F9
:102B600029F0809192028823E9F006C0F901ED571F
:102B7000FD4F90819423B1F086E0829FF001839F06
:102B8000F00D1124E60FF71FEE0FFF1FEB5EFE4F57
:102B9000808191818D939C93F901ED57FD4F808148
:102BA000482B06C0F901ED57FD4F40958081482321
:102BB00040830895CF93DF93CDB7DEB72B970FB641
:102BC000F894DEBF0FBECDBF942F4F83252F5887BB
:102BD00069877A878B874A855B85452B21F02F3F54
:102BE00009F59F3FF9F4DE01119686E0FD0111928F
:102BF0008A95E9F785E0FE01379601900D928A9556
:102C0000E1F749815A816B817C818D819E810E948F
:102C10001D1D2B960FB6F894DEBF0FBECDBFDF9102
:102C2000CF910895CE0107960E949E15DCCFCF93D9
:102C3000DF931F92CDB7DEB7882309F403C1682F55
:102C40008238C1F40E949B1481FDFCC069E380912D
:102C50000301909104010E949A210E9445202FEFC8
:102C600081EE94E0215080409040E1F700C00000E8
:102C700069E319C0833811F50E949B1480FDE2C0FE
:102C800063E580910301909104010E949A210E94C2
:102C900045202FEF81EE94E0215080409040E1F7F5
:102CA00000C0000063E580910301909104010E943F
:102CB000A5210F90DF91CF910C9445208438C1F469
:102CC0000E949B1482FDBEC067E480910301909135
:102CD00004010E949A210E9445202FEF81EE94E08A
:102CE000215080409040E1F700C0000067E4DBCF56
:102CF0008CEF860F813A70F4862F69830E946B26D1
:102D0000698181119FC080910301909104010E940B
:102D10009A21CFCF80E2860F883048F4677081E037
:102D200001C0880F6A95EAF70E947B20C2CF8BE52D
:102D3000860F833088F4653A29F0663A31F083E8EB
:102D400090E005C081E890E002C082E890E00F903A
:102D5000DF91CF910C94BD1488E5860F853108F082
:102D600071C0683A61F1693A69F16A3A71F16B3A96
:102D700079F16C3A81F16B3B89F16C3B91F16D3AE1
:102D800099F1603BA1F16E3AA9F16F3AB1F1613B63
:102D9000B9F1623BC1F1633BC9F1643BD1F1653BE1
:102DA000D9F1663BE1F1673BE9F1683BF1F1693B41
:102DB000F9F16A3B09F43FC080E090E03EC082EE4A
:102DC00090E03BC089EE90E038C08AEE90E035C0DC
:102DD00085EB90E032C086EB90E02FC083EB90E073
:102DE0002CC084EB90E029C087EB90E026C08CECEF
:102DF00090E023C08DEC90E020C083E891E01DC0FE
:102E00008AE891E01AC082E991E017C084E991E074
:102E100014C081E292E011C083E292E00EC084E22D
:102E200092E00BC085E292E008C086E292E005C025
:102E300087E292E002C08AE292E00F90DF91CF91A8
:102E40000C94D3140F90DF91CF910895882309F447
:102E50005BC0682F823879F40E949B1481FF54C0B4
:102E600069E380910301909104010E949A210E94DC
:102E7000452069E310C08338B1F40E949B1480FFA1
:102E800043C063E580910301909104010E949A215F
:102E90000E94452063E580910301909104010E9406
:102EA000A5210C944520843879F40E949B1482FF5C
:102EB0002BC067E480910301909104010E949A2144
:102EC0000E94452067E4E7CF8CEF860F813A18F324
:102ED00080E2860F883048F4677081E001C0880F77
:102EE0006A95EAF70E948120DCCF8BE5860F83305C
:102EF00020F480E090E00C94BD14685A653120F411
:102F000080E090E00C94D3140895882321F00E946F
:102F10007B200C9445200895882321F00E94812075
:102F20000C94452008958F929F92AF92BF92CF92BA
:102F3000DF92EF92FF920F931F93CF93DF931F9235
:102F4000CDB7DEB77C01C72EFC01058102950F705D
:102F50001281112321F069830E949820698169837D
:102F60000E943E206981882381F0112371F080E264
:102F7000860F883050F082E00E9427200E943E2079
:102F800091E0D82ED926698101C0D12CAC2CA29415
:102F90008FE0A822B12CF501E159FF4F0C94A1312B
:102FA0008C2D807F0C2D0F70882311F00295007FEF
:102FB0001123C1F0002309F4D2C180E2860F8830CA
:102FC00010F0611105C0802F69830E947B2004C02E
:102FD000802F69830E948B20698169830E9445202C
:102FE0006981BDC1862F69830E94261769810023EC
:102FF00009F40EC280E2860F883010F0611104C01F
:10300000802F0E94812003C0802F0E9491200E9467
:103010004520FEC19C2D907F8C2D8F70903211F039
:103020008295807F662319F06130B1F01EC01123B4
:1030300049F0002309F44BC1013009F048C10E9456
:10304000AB20E6C1002319F0013009F4E1C1898306
:103050000E94AE20898141C1112321F0023008F085
:10306000D7C135C10111D4C138C1112321F00023CA
:1030700009F42DC174C1002309F42FC181C18C2D25
:1030800086958695837090E0009719F0019761F01E
:10309000BFC1112321F0862F9C2D937002C080E0C8
:1030A00090E00E94BD14C4C1112321F0862F9C2DF5
:1030B000937002C080E090E00E94D314B9C1112344
:1030C000F9F0653F51F0663F71F0643FA9F48091DB
:1030D000A5039091A60381600BC08091A5039091F8
:1030E000A603826005C08091A5039091A603846029
:1030F0009093A6038093A503862F0E944A231EC0A7
:10310000653F51F0663F71F0643FA9F48091A503DB
:103110009091A6038E7F0BC08091A5039091A6038A
:103120008D7F05C08091A5039091A6038B7F90931E
:10313000A6038093A503862F0E94B2230E94372402
:1031400077C18C2D837009F052C011116DC1862F8B
:10315000829586958770880F880F962F9F70892E8D
:10316000912CA12CB12C082E04C0880C991CAA1CEF
:10317000BB1C0A94D2F764FF14C00FE010E020E0FB
:1031800030E0B901A80104C0440F551F661F771F26
:103190008A95D2F7CB01BA0160957095809590958C
:1031A00003C060E070E0CB012C2D2695269523709E
:1031B00030E02230310569F02330310589F068298B
:1031C00079298A299B292130310571F00E94601EDE
:1031D0002BC1682979298A299B290E94721E24C142
:1031E0000E94601EC501B4010E944E1E1DC1112324
:1031F00019F08C2D817001C08695882309F414C1C3
:10320000862F829586958770880F880F962F9F70DE
:10321000892E912CA12CB12C082E04C0880C991C4D
:10322000AA1CBB1C0A94D2F764FF14C00FE010E084
:1032300020E030E0B901A80104C0440F551F661F0B
:10324000771F8A95D2F7CB01BA016095709580956A
:10325000909503C060E070E0CB012C2D269526955B
:103260002370422F50E04230510569F04330510540
:1032700089F0682979298A299B294130510571F003
:103280000E94251FD1C0682979298A299B290E947B
:10329000371FCAC00E94251FC501B4010E94131F19
:1032A000C3C0862F90E0FC01E05EF109E531F10535
:1032B00008F051C0E158FF4F0C94A131062F0F7058
:1032C0008C2D8F71112331F00E94AC1E802F0E9433
:1032D00085179EC00E94CD1E802F0E948C1798C01B
:1032E000112339F0011194C08C2D8F710E94F21EB0
:1032F0008FC0023008F08CC0F7CF112339F08C2D2D
:103300008F710E94AC1E84C01123C9F38C2D8F7164
:103310000E94CD1E7DC0112329F08C2D8F710E943B
:10332000971E76C00E94921E73C0112351F01C2D6F
:103330001F71812F0E94AC1E63E0812F0E941E200E
:1033400067C081E00E942720023008F461C082E05B
:103350000E9427205DC0112331F0002381F2862FC7
:103360000E94171655C0002389F2693349F45FEFB4
:1033700077EE83E0515070408040E1F700C00000DC
:10338000862F0E94261744C04C2D4F70C7010E9403
:1033900013070E94C11D4CC0623F99F128F4603FA1
:1033A00049F0613FE1F020C0643FA1F050F0653F7B
:1033B00059F01AC0112339F19091920281E08927C6
:1033C00006C081E018271DC011111DC081E0809347
:1033D000920219C0111117C01092920214C000235A
:1033E00081F0111110C0E8CF002359F0862F6983B6
:1033F000112319F00E94171602C00E942617698136
:1034000002C0109392024C2D4F70C7010E94900A87
:1034100098E0A916B10441F05CF0FAE0AF1AB108E7
:1034200022E0A216B10420F40E949B140E948E0A8E
:10343000DD20F1F00E941A2080FD1AC0F7011282EF
:103440000E9414200E94AC1EC7010E94461A0E94CE
:1034500014200F90DF91CF911F910F91FF90EF906B
:10346000DF90CF90BF90AF909F908F900C94CD1E27
:103470000F90DF91CF911F910F91FF90EF90DF9010
:10348000CF90BF90AF909F908F9008950F931F9310
:10349000CF93DF93EC01888199812B813C81232B91
:1034A000B9F09F3F11F48F3F99F0CE010E94880739
:1034B000882371F0688179818A810E94F11F8C01D3
:1034C0000E94491F0E944B1EB801CE010E94931713
:1034D000DF91CF911F910F9108950E9498200E9433
:1034E000A82080910301909104010E94B0210E94C4
:1034F00045200E94D0240E94372480E090E00E9462
:10350000BD1480E090E00C94D3140E9488200C94A9
:103510006D1A0E94E61FE92FE295EF70F0E03297F6
:10352000EE30F105B0F4EC56FF4F0C94A131803F22
:1035300091F018F4803E68F40EC0843F51F40BC043
:10354000803E48F0813F29F406C093FB882780F92C
:10355000089580E0089581E00895CF93DF9300D02F
:1035600000D01F92CDB7DEB70F900F900F900F9045
:103570000F90DF91CF910895CF93DF9300D000D0CB
:1035800000D0CDB7DEB726960FB6F894DEBF0FBEDB
:10359000CDBFDF91CF9108951F93CF93DF93C0915B
:1035A000930216E080919402C81799F0D0E01C9F16
:1035B000F0011D9FF00D1124EB56FD4F408151810C
:1035C00062817381848195810E94BC1A2196C770A3
:1035D000E9CFDF91CF911F9108954091C50250919D
:1035E000C6026091C7027091C8028091C902909191
:1035F000CA020C94BC1A8091CA0282958F7009F09D
:1036000054C08091C702882309F44FC0809193026F
:10361000A09194026091C5027091C6024091C802C7
:103620005091C902B6E08A1709F43FC090E04115F5
:103630005105C1F17F3F11F46F3FA1F1B89FF00137
:10364000B99FF00D1124EB56FD4F218172132AC052
:103650002081621327C02281211124C0238134815B
:103660002417350710F421503109241B350B283C51
:103670003105C0F42091CA022F7020612093CA0244
:1036800026E0289FF001299FF00D1124E656FD4FFA
:1036900080818F708061808385EC92E00E94461A61
:1036A0000C94CC1A01968770BECF0895CF92DF920A
:1036B000EF92FF920F931F93CF93DF93CDB7DEB7B7
:1036C00062970FB6F894DEBF0FBECDBF8C0185E0C8
:1036D000F801DE011D9601900D928A95E1F7D8015F
:1036E0004C9111965C91119712966C9112971396CA
:1036F000CD90DC9014973091C5027091C6028091F4
:10370000C8029091C902009709F46BC17F3F19F478
:103710003F3F09F466C1E090C702EE2009F4C0C043
:103720002091CA02C816D90628F0F601E81BF90B49
:10373000CF0104C0809590958C0D9D1DFF24F394BE
:10374000883C910578F0F12C207F09F0C6C07C2DD3
:10375000D98AC88A89890E94AD1A85EC92E00E94B4
:10376000461AB1C0822F807F09F046C0751314C07D
:10377000341312C0611110C02F7020612093CA024F
:103780000E94ED1A85EC92E00E94461A8091CA02CE
:10379000D80115968C932EC0CD2819F15F3F11F4F6
:1037A0004F3FF9F0F62E61111CC0809193022091D9
:1037B000940236E0821709F45AC090E0389FF00175
:1037C000399FF00D1124EB56FD4F7181571306C040
:1037D0007081471303C07281711103C00196877015
:1037E000E9CFF62E662309F418C18091CA028160E0
:1037F0008093CA02F12C11C1751308C0341306C09E
:10380000611104C08091CA02D801C3C04D875E8790
:103810008D859E856A8B0E94891A6A898823E1F1C9
:103820006623D1F12091CA02822F82958F7090E099
:10383000029774F08091C5029091C60298878F8399
:103840001986DB86CA862C87CE0107960E94461A07
:1038500086E0F801A5ECB2E001900D928A95E1F7BF
:103860000E94FB1A0E94ED1AFF24F394D6C04D87E4
:103870005E878D859E850E94E61F292F22952F70D9
:1038800030E0223031050CF0BCC09F7009F0B6C0AA
:10389000805E883008F4C1C0C8010E94461AE4CF97
:1038A000C816D90608F453C0F601E81BF90BCF017E
:1038B000883C910508F450C0F12C7C2DD98AC88A27
:1038C00089890E94AD1AE5ECF2E086E0DF011D92E5
:1038D0008A95E9F70E94ED1AA0C0751314C034133D
:1038E00012C0611110C08091CA02F8018583C8011D
:1038F0000E94461A86E0E5ECF2E0DF011D928A950F
:10390000E9F7FE2C8AC04D875E878D859E856A8B80
:103910000E94891A6A89882309F4BECF662309F4B4
:10392000BBCF2091CA02822F82958F7090E00297C0
:103930000CF48ECF8091C5029091C6029A83898340
:103940001B82DD82CC822E83CE0101967FCF8095B3
:1039500090958C0D9D1DACCFF62E662309F49CCF5F
:1039600075132EC034132CC02091CA0220FD1FC035
:10397000822F82958F70D9F0D80115962C931597C8
:103980008F3049F08F5F982F9295907F822F8F70A4
:10399000892B15968C93C8010E94461A86E0F8017F
:1039A000A5ECB2E001900D928A95E1F793CF86E005
:1039B000F801A5ECB2E001900D928A95E1F72DC0D7
:1039C0004D875E878D859E850E94891A811140CF23
:1039D0008091CA0281608093CA02C8010E94461A7F
:1039E0001CC0662309F458CF4D875E878D859E8560
:1039F0000E94891A882309F44FCF2ACF811148CF1A
:103A00000CC0243031050CF047CF9F7009F440CF33
:103A1000F8019581907F09F03BCF8F2D62960FB60C
:103A2000F894DEBF0FBECDBFDF91CF911F910F91F4
:103A3000FF90EF90DF90CF9008951F93CF93DF9387
:103A4000CDB7DEB72C970FB6F894DEBF0FBECDBF53
:103A50004F83588769877A878B879C87CE01079623
:103A60000E94561B882369F08F8198852A853B85A3
:103A7000232BF1F19F3F09F063C08F3F09F060C035
:103A800037C086E0FE013796DE01119601900D9257
:103A90008A95E1F76F817885EA85FB85309741F15A
:103AA0007F3F11F46F3F21F12091940230E0C90172
:103AB0000196877099274091930250E084179507EB
:103AC00009F447C069837A83FD83EC8396E0929F73
:103AD000D001939FB00D1124AB56BD4FFE0131961E
:103AE00001900D929A95E1F7809394020E94CC1A6E
:103AF00016E080919302909194028917C1F1189F6A
:103B0000C00111248B569D4F0E94561B882379F1CA
:103B1000E09193021E9FF0011124EB56FD4F40816E
:103B2000518162817381848195810E94BC1A809148
:103B3000930290E001968770992780939302D9CFE2
:103B40004F81588569857A858B859C850E94BC1A32
:103B5000CFCF0E94851A1092940210929302E5EC46
:103B6000F2E086E0DF011D928A95E9F7C1CF2C963D
:103B70000FB6F894DEBF0FBECDBFDF91CF911F917E
:103B80000895EF92FF920F931F93CF93DF938C01D1
:103B9000892B09F46CC0F12CEE24E394E801219602
:103BA000F8018491843740F4843008F051C08130AA
:103BB00081F0823019F15BC0853709F444C0A8F167
:103BC0009CE7980F903708F052C08F770E94261715
:103BD00041C00E5F1F4FFE01C49180E28C0F883000
:103BE00048F4C7708E2D01C0880FCA95EAF70E946D
:103BF0009B2014C08C2F0E9417162DC00E5F1F4FE4
:103C0000FE01C49180E28C0F883058F4C7708E2D6D
:103C100001C0880FCA95EAF70E94A1200E944520A2
:103C20001AC08C2F0E94261716C00E5F1F4FFE0170
:103C3000C491CC2381F08FE99FE00197F1F700C098
:103C40000000C150F6CF0E5F1F4FFE01F49003C07D
:103C50000E9417168E018F2D882309F49FCFEFE95C
:103C6000FFE03197F1F700C000008150F5CFDF9100
:103C7000CF911F910F91FF90EF90089508950E94AA
:103C80003E1E60930603709307038093080390938E
:103C900009030C946D1A08950C943F1E0F931F9303
:103CA0000091060310910703209108033091090346
:103CB000602B712B822B932B1F910F910C943F1E25
:103CC0000F931F930091060310910703209108039F
:103CD0003091090360237123822393231F910F9155
:103CE0000C943F1E0F931F9300910603109107033E
:103CF00020910803309109036027712782279327B9
:103D00001F910F910C943F1E0C9445070E94841E36
:103D1000609302037093030380930403909305035D
:103D20000C946D1A60E070E0CB010C94861E0F932A
:103D30001F9341E050E060E070E08A019B0104C005
:103D4000000F111F221F331F8A95D2F7C901B80136
:103D50001F910F910C94861E0F931F9341E050E02A
:103D600060E070E004C0440F551F661F771F8A95FE
:103D7000D2F78091020390910303A0910403B091C4
:103D800005038A019B01082B192B2A2B3B2BC90108
:103D9000B8011F910F910C94861E0F931F9341E061
:103DA00050E060E070E004C0440F551F661F771FAD
:103DB0008A95D2F740955095609570958091020351
:103DC00090910303A0910403B09105038A019B0124
:103DD000082319232A233B23C901B8011F910F91FE
:103DE0000C94861E0F931F9341E050E060E070E05A
:103DF00004C0440F551F661F771F8A95D2F7809124
:103E0000020390910303A0910403B09105038A017A
:103E10009B01082719272A273B27C901B8011F91B1
:103E20000F910C94861E0F931F9300910203109123
:103E300003032091040330910503602B712B822B27
:103E4000932B1F910F910C94861E0F931F9300913B
:103E500002031091030320910403309105036023B2
:103E60007123822393231F910F910C94861E0F932D
:103E70001F930091020310910303209104033091DA
:103E8000050360277127822793271F910F910C94B8
:103E9000861E0895292F220F920F990F890FA82FA0
:103EA000A695A695A695877051E001C0550F8A95F5
:103EB000EAF785E0A89FD001112420E030E070E00F
:103EC000F901EA0FFB1FE553FD4F4081CB01022EA4
:103ED00002C0969587950A94E2F78170992781959B
:103EE00084278523842780832F5F3F4F253031052A
:103EF00039F70895292F220F920F990F890F682FF4
:103F0000669566956695982F977085E0689FB001D5
:103F1000112440E050E080E0FA01E60FF71FE5537E
:103F2000FD4F208130E0092E02C0369527950A9476
:103F3000E2F721703327042E01C0220F0A94EAF71A
:103F4000822B4F5F5F4F4530510531F70895CF9277
:103F5000DF92EF92FF920F931F93CF93DF938C0129
:103F6000C0900603D0900703E0900803F090090387
:103F70008091020390910303A0910403B091050383
:103F8000C82AD92AEA2AFB2ACFE1D0E0D701C60104
:103F90000C2E04C0B695A795979587950A94D2F7ED
:103FA00080FF06C0B8018C2F0E94AB0A019721F454
:103FB000219760F780E001C08C2FDF91CF911F9196
:103FC0000F91FF90EF90DF90CF900895CF93DF9304
:103FD000EC010E94A71FBE010E94AB0ADF91CF91A6
:103FE00008951F93CF93DF93EB0190919102992352
:103FF00021F0CB010E94E61F13C0882349F0CB01BA
:104000000E94A71F182F682FCE010E944A1F04C0CC
:10401000CB010E947A1F182FBE01812F0E94AB0A8C
:10402000DF91CF911F91089580910A038595859521
:104030008595089580910A038770089598E0899F77
:1040400090011124262B20930A030C94AC1E20917E
:104050000A038095822380930A03982F977069F44E
:1040600030E0482F082E000C550B2417350729F097
:104070008595859585950C94CD1E089590910A039C
:10408000977081E009F480E00895E0910301F091D8
:10409000040180912E038083E0910301F0910401DB
:1040A000908180912D03892B8083E0910301F09111
:1040B0000401908180912C03892B808380910B03D4
:1040C000882381F0E0910301F09104019081892B14
:1040D000808380910301909104010E943E2181110F
:1040E00010920B0380910301909104010C94A7148A
:1040F00080912E03089590912E03892B80932E0397
:104100000895809590912E03892380932E0308951E
:1041100010922E03089590912D03892B80932D03E7
:104120000895809590912D03892380932D03089500
:1041300010922D03089590912C03892B80932C03CA
:104140000895809590912C03892380932C030895E2
:1041500010922C03089580930B03089510920B0383
:104160000895CF92DF92EF92FF926C01EE24FF242C
:10417000C114D104E104F10421F0C701B60120E12A
:1041800001C020E0C72ED82EE92EFF24C114D1048F
:10419000E104F10419F0285FC701B6016B017C014D
:1041A00054E0F694E794D794C7945A95D1F7C11484
:1041B000D104E104F10419F02C5FC701B6016B01D1
:1041C0007C0142E0F694E794D794C7944A95D1F7DE
:1041D000C114D104E104F10419F02E5FC701B60146
:1041E000DC01CB01B695A79597958795892B8A2BEE
:1041F0008B2B09F02F5F822FFF90EF90DF90CF90F5
:1042000008956DEE7EEF80E090E00E94D93160E08D
:1042100082E090E00E94BB3160E083E090E00E9489
:10422000BB3160E084E090E00E94BB3160E085E05B
:1042300090E00E94BB3140E050E0BA0188E090E09D
:104240000C94CD3180E090E00E94B53121E08D3EAC
:104250009E4F09F020E0822F089582E090E00C94B8
:10426000A73183E090E00C94A73184E090E00C94B7
:10427000A731682F84E090E00C94BB31FC013196AB
:104280009C01205E3F4F80E0919191118F5FE2177A
:10429000F307D1F708959C01FC0132969FEF80E06F
:1042A0004191461789F09F3F19F4411101C0982FA1
:1042B0008F5F8E31A9F79F3F39F0F901E90FF11DAA
:1042C00097FDFA95628308950895FC0132968096D1
:1042D0002081261301C010823196E817F907C1F733
:1042E0000895262F2695269526952F3168F4FC01F2
:1042F000E20FF11D677021E030E001C0220F6A95E6
:10430000EAF78181282B21830895262F269526956B
:1043100026952F3170F4FC01E20FF11D677021E04A
:1043200030E001C0220F6A95EAF7209581812823A9
:104330002183089520911401222329F02091AB03B9
:1043400027FD0C9471210C944B2120911401222300
:1043500029F02091AB0327FD0C9485210C94652155
:10436000FC01319680961192E817F907E1F708955C
:104370008091B103843039F11092300320E488E158
:1043800090E00FB6F894A895809360000FBE20933C
:10439000600080E00E948E0A83B7817F846083BFC3
:1043A00083B7816083BF7894889583B78E7F83BFFE
:1043B0000FB6F894A89580916000886180936000A2
:1043C000109260000FBE08950895CF930E942005BB
:1043D0000E946D050E94E421C0E08C2F0E944F06D0
:1043E000811104C0CF5FCE30C1F701C081E0CF9111
:1043F00008950E94851A0E949B140C948E0A1F92A5
:104400000F920FB60F9211248F939F93AF93BF9388
:1044100080913003811113C08091A7039091A8036C
:10442000A091A903B091AA034196A11DB11D80934B
:10443000A7039093A803A093A903B093AA03BF91E5
:10444000AF919F918F910F900FBE0F901F90189575
:1044500082E084BD93E095BD9AEF97BD80936E0096
:1044600008952FB7F8948091A7039091A803A09185
:10447000A903B091AA032FBF0895CF92DF92EF92C4
:10448000FF920F931F932FB7F8944091A703509179
:10449000A8036091A9037091AA032FBF6A017B0151
:1044A000EE24FF248C0120E030E0C016D106E206A5
:1044B000F30610F4415051099A01281B390BC90128
:1044C0001F910F91FF90EF90DF90CF900895789417
:1044D0001F920F920FB60F9211248F939F93AF9359
:1044E000BF938091A7039091A803A091A903B091D5
:1044F000AA030196A11DB11D8093A7039093A80361
:10450000A093A903B093AA03BF91AF919F918F91FC
:104510000F900FBE0F901F9018950E94292BF894B2
:104520002FEF87EA91E6215080409040E1F700C0EC
:10453000000087E090EBDC018093BA039093BB030B
:10454000A093BC03B093BD039CE088E10FB6F89440
:10455000A895809360000FBE90936000FFCF0E94EB
:104560002221811102C00E9401210E942D218093ED
:104570002F030E94352190E09093AC038093AB030E
:104580000E943121682F70E080E090E00C944C1E76
:104590008091340380FF0BC06091080185E0689F23
:1045A000B001112475956795759567952BC081FFAE
:1045B00009C06091080185E0689FB00111247595DC
:1045C000679520C082FF07C06091080185E0689F61
:1045D000B001112417C0909135039923D1F0609157
:1045E0000701961788F72091080185E0289F900120
:1045F0001124929FA001939F500D112470E0CA01D5
:104600000E948D316038710540F46115710539F0F3
:1046100002C065E070E0862F08958FE7089581E07D
:1046200008958091340380FF08C06091060170E016
:10463000759567957595679521C081FF06C0609156
:10464000060170E07595679519C082FF04C06091FE
:10465000060170E010C0909135039923C1F060917C
:1046600005019617A0F780910601899FC0011124CA
:1046700070E00E948D316038710528F46115710574
:1046800021F0862F08958FE7089581E0089561E075
:1046900070E0F4CF803F21F40E94C822819504C0CD
:1046A000813F29F40E94C822809338030895823FF5
:1046B00021F40E94C822819504C0833F29F40E94FE
:1046C000C822809337030895893F19F40E9411236B
:1046D00005C08A3F31F40E941123819580933903EC
:1046E00008958B3F21F40E941123819504C08C3FD3
:1046F00029F40E94112380933A030895843F21F402
:1047000080913603816017C0853F21F48091360384
:10471000826011C0863F21F48091360384600BC013
:10472000873F21F480913603886005C0883F31F4CB
:104730008091360380618093360308958D3F21F484
:104740008091340381600BC08E3F21F4809134034B
:10475000826005C08F3F29F4809134038460809388
:1047600034030895803F39F48091380387FF6CC08B
:104770001092380369C0813F29F4809138031816DC
:10478000BCF362C090913703823F29F497FF5CC06D
:104790001092370359C0833F19F41916CCF354C053
:1047A000893F41F48091390318160CF04DC01092E6
:1047B00039034AC08A3F29F48091390387FF44C0F6
:1047C000F6CF8B3F39F480913A0387FF3DC01092BA
:1047D0003A033AC08C3F29F480913A031816BCF38F
:1047E00033C0843F21F4809136038E7F17C0853F0C
:1047F00021F4809136038D7F11C0863F21F4809192
:1048000036038B7F0BC0873F21F480913603877F6F
:1048100005C0883F31F4809136038F7E8093360344
:1048200013C08D3F21F4809134038E7F0BC08E3FE7
:1048300021F4809134038D7F05C08F3F29F480914E
:1048400034038B7F809334038091370381110EC032
:104850008091380381110AC080913903811106C00B
:1048600080913A03811102C010923503089586E3C6
:1048700093E00E94B2140E943122909332038093FD
:10488000310308951F93CF93DF938091310390916B
:1048900032030E943D22AC0190913503992321F00F
:1048A0002091090130E006C0209133038AE0289F5F
:1048B000900111244217530708F46EC0809137030A
:1048C000C0913803D091390310913A03811107C088
:1048D000C1115EC0D1115CC011115AC05DC09F3FB3
:1048E00019F09F5F90933503181624F40E94C82294
:1048F000809337038091370387FF05C00E94C82249
:104900008195809337031C1624F40E94C82280935B
:1049100038038091380387FF05C00E94C822819523
:104920008093380340913703442379F03091380362
:10493000332359F025EB4203A00111245093370390
:104940003203C0011124909338031D1624F40E94F1
:104950001123809339038091390387FF05C00E949A
:104960001123819580933903111624F40E94112399
:1049700080933A0380913A0387FF05C00E94112378
:10498000819580933A03DF91CF911F910C94372446
:104990009F3F09F0A6CFAECFDF91CF911F91089531
:1049A000E6E3F3E085E0DF011D928A95E9F71092D6
:1049B0003503109234030895833081F128F4813057
:1049C00059F08230D1F00895853009F449C0B8F12A
:1049D000863009F456C0089580913303262F30E0C5
:1049E000280F311D2F3F310524F4680F60933303E6
:1049F00008958FEF80933303089580910901262F46
:104A000030E0280F311D2F3F310524F4680F6093EB
:104A1000090108958FEF809309010895809108019D
:104A2000262F30E0280F311D2F3F310524F4680F69
:104A30006093080108958FEF809308010895809195
:104A40000701262F30E0280F311D2F3F310524F4B8
:104A5000680F6093070108958FEF80930701089511
:104A600080910601262F30E0280F311D2F3F3105A0
:104A700024F4680F6093060108958FEF8093060178
:104A8000089580910501262F30E0280F311D2F3F1A
:104A9000310524F4680F6093050108958FEF80932A
:104AA00005010895833011F128F4813049F08230F6
:104AB00091F00895853081F120F18630C1F108959B
:104AC00080913303681720F4861B80933303089585
:104AD00010923303089580910901681720F4861B12
:104AE00080930901089510920901089580910801A9
:104AF000681720F4861B809308010895109208011E
:104B0000089580910701681720F4861B80930701A0
:104B1000089510920701089580910601681720F406
:104B2000861B8093060108951092060108958091D6
:104B30000501681720F4861B8093050108951092E3
:104B4000050108950F931F93873208F04DC08E31F1
:104B500008F093C0803109F47DC008F5873009F46E
:104B60006BC068F4863009F0A3C080912F03817F69
:104B70008E7F80932F0381E080933C039AC08B301B
:104B800009F48FC08E3009F093C080912F0382FB0F
:104B9000222720F991E0922790FB82F964C08631A8
:104BA00009F47FC088F4813109F082C00E94851A1F
:104BB0008091AB0387FB222720F991E0922790FB9D
:104BC00087F98093AB036DC0893109F46AC08B31DA
:104BD00009F06EC080912F0381FB222720F991E01C
:104BE000922790FB81F93FC0883309F45AC050F4F2
:104BF000893209F458C0853309F455C0873209F465
:104C000052C056C0833409F44EC028F48A3308F4E5
:104C10004FC0895333C0883409F04AC00E94851AB6
:104C20000FEF13ED20E3015010402040E1F700C0EA
:104C300000000E948D2235C080912F03982F9095FF
:104C4000917090FB80F980932F0391112AC0897F86
:104C5000877F10C080912F0383FB222720F991E0EA
:104C6000922790FB83F980932F039923D1F08091B1
:104C70002F03816080932F0314C08D5141E050E0D9
:104C800060E070E08A019B0104C0000F111F221F29
:104C9000331F8A95D2F7C901B8010E944C1E0E94A9
:104CA000851A81E006C061E070E080E090E0F5CF19
:104CB00080E01F910F91089580E0089580E00895AD
:104CC0008E518A3030F4E82FF0E0E354FE4F8081BB
:104CD000089580E00895CF93C82F80913C038130E0
:104CE00079F018F08230E9F185C0E0910301F0918C
:104CF00004018081813169F0823209F07DC009C0F0
:104D0000E0910301F09104018081813111F0823240
:104D100061F48C2F0E945C26811104C08C2F0E94AC
:104D2000A2251DC081E090E01AC08C2F0E945E2653
:104D3000811114C0C43179F048F4CB3079F0C0311E
:104D400009F05EC082E080933C0308C0C93219F0CC
:104D5000C83321F055C010923C0352C081E08170ED
:104D600051C0C93279F108F5C43161F1A0F4C730FE
:104D700009F044C01092330384E180930901C09389
:104D800008018CE38093070188E08093060188E2A4
:104D90008093050133C082EE8C0F863078F58C2F1E
:104DA0000E94602680933B0329C0CE34E9F020F4B2
:104DB000CB3421F56AE013C0C13579F0C235F1F486
:104DC00061E00DC080913B03882319F010923B03F2
:104DD00015C081E080933C0315C061E006C080915E
:104DE0003B030E94DC240AC06AE080913B030E94DE
:104DF000522504C010923C0380E004C081E002C050
:104E000080E0ADCFCF91089580915D0308950F9319
:104E10001F93CF93DF9300D01F92CDB7DEB78C01E5
:104E20000E947729823011F0843019F593E099833C
:104E30001B830A839093E9008FEF9091E8008150E3
:104E400095FD06C095ED9A95F1F700008111F5CF1B
:104E50008091E80085FF0DC040E050E063E070E025
:104E6000CE0101960E9494298091E8008E7780936C
:104E7000E8000F900F900F90DF91CF911F910F914D
:104E80000895CF93DF9300D01F92CDB7DEB7209166
:104E9000B103243031F522E02983805891099B83A6
:104EA0008A8383E08093E9008FEF9091E80081503E
:104EB00095FD06C095ED9A95F1F700008111F5CFAB
:104EC0008091E80085FF0DC040E050E063E070E0B5
:104ED000CE0101960E9494298091E8008E778093FC
:104EE000E8000F900F900F90DF91CF910895CF932E
:104EF000DF93EC010E947729823011F08430F9F4BD
:104F000082E08093E9009FEF8091E800915085FD59
:104F100006C085ED8A95F1F700009111F5CF8091DB
:104F2000E80085FF0CC040E050E065E070E0CE0195
:104F30000E9494298091E8008E778093E800DF91A9
:104F4000CF910895CF93DF93EC010E9477298230AF
:104F500019F0843009F047C0809114018823E1F0F2
:104F60008091AB0387FF18C084E08093E9008FEF46
:104F70009091E800815095FD06C095E19A95F1F772
:104F800000008111F5CF8091E80085FF2CC040E042
:104F900050E060E270E017C081E08093E9008FEF9D
:104FA0009091E800815095FD06C095ED9A95F1F736
:104FB00000008111F5CF8091E80085FF14C040E02A
:104FC00050E068E070E0CE010E9494298091E800F2
:104FD0008E778093E80080E2FE01ADE3B3E00190BC
:104FE0000D928A95E1F7DF91CF9108958091B003FA
:104FF000811109C00E94292B0E94862B8091E2001A
:1050000084608093E20008951092B003089508959B
:1050100008950C94F92142E061EC81E00E94A32AFA
:1050200042E061EC82E00E94A32A42E061EC83E06E
:105030000E94A32A42E261EC84E00C94A32A8091AE
:10504000B303833009F455C030F4813071F08230FD
:1050500009F48EC008958A3009F47AC08B3009F4BF
:1050600060C0893009F09CC020C08091B203813AB1
:1050700009F096C08091E800877F8093E8008091D6
:10508000B6039091B703892B21F460E28DE393E09E
:1050900003C060E080E090E070E00E94DF29809132
:1050A000E8008B778093E80008958091B203813205
:1050B00009F076C08091B6039091B703009719F07C
:1050C000039709F06DC08091E800877F8093E80026
:1050D0008091E80082FD05C08091B1038111F8CF75
:1050E0005FC08091F10080935D038091E8008B7731
:1050F00053C08091B203813A09F052C08091B60347
:105100009091B703892B09F04BC08091E800877F0D
:105110008093E8008091E80080FFFCCF809114012B
:1051200036C08091B2038132D9F58091B603909157
:10513000B703892BA9F58091E800877F8093E80069
:105140000E94D82A8091B403809314010C94851A8C
:105150008091B203813221F58091E800877F8093AE
:10516000E8000E94D82A8091B50380935E030895D9
:105170008091B203813AA1F48091E800877F809307
:10518000E8008091E80080FFFCCF80915E0380936F
:10519000F1008091E8008E778093E8000C94D82A83
:1051A000089584B7877F84BF0FB6F894A89580913F
:1051B0006000886180936000109260000FBE80E8FC
:1051C00080936100109261000E94EA140E94292BD2
:1051D0000E94862B8091E20084608093E2007894A4
:1051E0000E94152E0E94EE148AE091E00E9496140F
:1051F0008091B103853069F40E94B8218091AF039A
:105200008823B1F30E94E521882391F30E947E292F
:10521000EFCF0E94F6140E949913EACF292F33276B
:1052200023303105C9F064F42130310581F022309A
:10523000310509F043C08DE690E02AEF36E042C028
:1052400021323105F1F02232310541F137C082E1DE
:1052500090E027E637E036C099278130910541F08C
:105260008230910541F0892B49F5E6EFF6E005C063
:10527000EEEDF6E002C0E6ECF6E0849190E09F01EE
:1052800021C064307105D0F4660F771FFB01ED5229
:10529000FE4F2081318189E090E014C064307105B7
:1052A00068F4FB01EE0FFF1FE553FE4F20813181B3
:1052B000FB01E953FE4F808190E004C080E090E064
:1052C00020E030E0FA013183208308950895CF93E0
:1052D000C82F0E946629C0935F03CF9108958091E3
:1052E000B103843011F081E0089582E00895809147
:1052F0005F03811102C00C946F29089580E189BD7C
:1053000082E189BD09B400FEFDCF8091D8008F7D78
:105310008093D8008091E00082608093E0008091CB
:10532000E00081FDFCCF0895CF92DF92EF92FF92D3
:105330000F931F93CF93DF93EC018B016A010E94BF
:10534000F72A811133C0C114D10439F0F6018081EC
:105350009181081B190BC80FD91FE12CF12C0115E5
:10536000110519F18091E80085FD16C08091E800D3
:105370008E778093E800C114D10449F0F601808152
:105380009181E80EF91EF182E08285E00FC00E9453
:10539000F72A882321F30AC089918093F1000150F4
:1053A0001109FFEFEF1AFF0ADACF80E0DF91CF910A
:1053B0001F910F91FF90EF90DF90CF900895209173
:1053C000B8033091B9032617370748F06115710506
:1053D00039F42091E8002E772093E80001C0B9014C
:1053E00040E061157105A9F12091B103222309F470
:1053F00043C0253009F442C02091E80023FD40C09D
:105400002091E80022FD32C02091E80020FFE9CF82
:105410004091F3002091F20030E0342BFC01CF01E9
:105420006115710559F02830310540F48191809360
:10543000F100615071092F5F3F4FF1CF41E02830FB
:10544000310509F040E02091E8002E772093E80034
:10545000C8CF4111C9CF0AC08091B103882361F040
:10546000853061F08091E80083FD0AC08091E800FA
:1054700082FFF2CF80E0089582E0089583E00895EE
:1054800081E008952091B8033091B90326173707BA
:1054900048F06115710539F42091E8002E772093CA
:1054A000E80001C0B901FC0120E06115710591F12E
:1054B0008091B103882309F440C0853009F43FC0CE
:1054C0008091E80083FD3DC08091E80082FD2FC0FF
:1054D0008091E80080FFE9CF2091F3008091F200F5
:1054E00090E0922B6115710559F08830910540F4D8
:1054F00024912093F1003196615071090196F2CF09
:1055000021E0089709F020E08091E8008E778093F1
:10551000E800CBCF2111CCCF0AC08091B103882302
:1055200061F0853061F08091E80083FD0AC08091D0
:10553000E80082FFF2CF80E0089582E0089583E0E2
:10554000089581E00895982F973058F59093E900D9
:10555000981739F07091EC002091ED005091F00017
:1055600003C0242F762F50E021FF19C03091EB00AB
:105570003E7F3093EB003091ED003D7F3093ED00A6
:105580003091EB0031603093EB007093EC0020938E
:10559000ED005093F0002091EE0027FF07C09F5FC1
:1055A000D3CF8F708093E90081E0089580E0089563
:1055B0008091B20387FF11C08091E80082FD05C091
:1055C0008091B1038111F8CF11C08091E8008B77F1
:1055D0000BC08091B103882349F08091E80080FFDF
:1055E000F8CF8091E8008E778093E80008952091AD
:1055F000E4003091E50095E64091EC00842F817045
:1056000040FF22C08091E80080FD1CC08091B10362
:10561000882391F0853091F08091EB0085FD10C0DA
:105620004091E4005091E5004217530729F39A0195
:10563000915011F784E0089582E0089583E0089581
:1056400081E0089580E008954091E80042FFDECFB8
:1056500008950E94972B0E949F2BE0EEF0E080813E
:1056600081608083E8EDF0E080818F77808319BCD2
:10567000A7EDB0E08C918E7F8C9380818F7E8083AC
:105680001092B00308950F931F93CF93DF930E945E
:10569000972B0E949F2BC8EDD0E088818F7788835D
:1056A00088818068888388818F7D888319BC109267
:1056B000B1031092AD031092AF031092AE0300EE4F
:1056C00010E0F80180818B7F8083888181608883EE
:1056D00042E060E080E00E94A32AE1EEF0E08081F9
:1056E0008E7F8083E2EEF0E0808181608083808124
:1056F00088608083F80180818E7F808388818061CB
:105700008883DF91CF911F910F910895E8EDF0E02C
:1057100080818F7E8083E7EDF0E0808181608083EF
:1057200084E082BF81E08093B0030C94432BE8EDCA
:10573000F0E080818E7F80831092E20008951092C5
:10574000DA001092E10008951F920F920FB60F92A7
:1057500011242F933F934F935F936F937F938F9376
:105760009F93AF93BF93EF93FF938091E10082FFEC
:105770000BC08091E20082FF07C08091E1008B7F27
:105780008093E1000E94142E8091DA0080FF1FC0F8
:105790008091D80080FF1BC08091DA008E7F8093BB
:1057A000DA008091D90080FF0DC080E189BD82E1DF
:1057B00089BD09B400FEFDCF81E08093B1030E9452
:1057C000F62705C019BC1092B1030E9404288091ED
:1057D000E10080FF19C08091E20080FF15C0809138
:1057E000E2008E7F8093E2008091E20080618093EE
:1057F000E2008091D80080628093D80019BC85E0D7
:105800008093B1030E9408288091E10084FF30C09A
:105810008091E20084FF2CC080E189BD82E189BDD6
:1058200009B400FEFDCF8091D8008F7D8093D80011
:105830008091E1008F7E8093E1008091E2008F7E75
:105840008093E2008091E20081608093E200809189
:10585000AD03882311F084E007C08091E30087FD49
:1058600002C081E001C083E08093B1030E94092857
:105870008091E10083FF29C08091E20083FF25C071
:105880008091E100877F8093E10082E08093B10303
:105890001092AD038091E1008E7F8093E1008091B2
:1058A000E2008E7F8093E2008091E200806180932D
:1058B000E20042E060E080E00E94A32A8091F000D4
:1058C00088608093F0000E940728FF91EF91BF91BC
:1058D000AF919F918F917F916F915F914F913F9188
:1058E0002F910F900FBE0F901F9018951F920F923F
:1058F0000FB60F9211242F933F934F935F936F93A3
:105900007F938F939F93AF93BF93CF93DF93EF9347
:10591000FF93C091E900CF708091EC00D82FD17037
:1059200080FDD0E81092E9008091F000877F80939D
:10593000F00078940E94BA2C1092E9008091F00057
:1059400088608093F000CD2BCF70C093E900FF9169
:10595000EF91DF91CF91BF91AF919F918F917F9107
:105960006F915F914F913F912F910F900FBE0F90CC
:105970001F9018951F93CF93DF93CDB7DEB7AA97EB
:105980000FB6F894DEBF0FBECDBFE2EBF3E088E0C8
:105990008E0F9091F10091938E13FBCF0E941F28E0
:1059A0008091E80083FF28C18091B2039091B303F6
:1059B000492F50E04A30510508F01EC1FA01EE555A
:1059C000FF4F0C94A131803821F0823809F014C1C6
:1059D00008C08091AE039091AF03992389F0826053
:1059E0000FC08091B6038F70873008F005C1809397
:1059F000E9008091EB0085FB882780F91092E9008F
:105A00009091E800977F9093E8008093F1001092C6
:105A1000F100D0C0282F2D7F09F0EEC0882319F0A7
:105A2000823061F0E9C08091B403813009F0E4C0B4
:105A3000933009F080E08093AF032EC08091B403CF
:105A400081112AC08091B6038F702FEF280F263066
:105A500008F0D2C08093E9002091EB0020FF1CC029
:105A6000933021F48091EB00806214C09091EB00A0
:105A700090619093EB0021E030E0A90102C0440F57
:105A8000551F8A95E2F74093EA001092EA00809150
:105A9000EB0088608093EB001092E9008091E800B1
:105AA000877F8093E8000E94D82AA6C08111A4C0F5
:105AB0001091B4031F778091E3008078812B80934D
:105AC000E3008091E800877F8093E8000E94D82A55
:105AD0008091E80080FFFCCF8091E3008068809394
:105AE000E300111102C082E001C083E08093B103A2
:105AF00083C08058823008F07FC08091B4039091B9
:105B0000B5038C3D53E0950779F583E08A838AE2FB
:105B100089834FB7F894DE01139620E03EE051E20E
:105B2000E32FF0E050935700E49120FF03C0E2958B
:105B3000EF703F5FEF708E2F90E0EA3010F0C79665
:105B400001C0C0968D939D932F5F243149F74FBFBD
:105B50008091E800877F8093E8006AE270E0CE01E0
:105B600001960E94DF2915C06091B6037091B703BA
:105B7000AE014F5F5F4F0E940E29BC01892BE1F1FE
:105B80009091E800977F9093E80089819A810E9424
:105B9000422A8091E8008B778093E8002DC08038FE
:105BA00059F58091E800877F8093E8008091AD03EC
:105BB0008093F1008091E8008E7773CF81111CC033
:105BC0009091B4039230C0F48091E800877F809375
:105BD000E8009093AD030E94D82A8091AD03811113
:105BE00006C08091E30087FD02C081E001C084E02F
:105BF0008093B1030E940B288091E80083FF0AC0C4
:105C00008091E800877F8093E8008091EB008062BC
:105C10008093EB00AA960FB6F894DEBF0FBECDBFFF
:105C2000DF91CF911F9108950895CF938091B10393
:105C30008823A1F0C091E900CF709091EC00892FEA
:105C4000817090FD80E8C82B1092E9008091E800F7
:105C500083FD0E94BA2CCF70C093E900CF910895C4
:105C60005058BB27AA270E94482E0C94F32F0E945D
:105C7000E52F38F00E94EC2F20F039F49F3F19F403
:105C800026F40C94BB2F0EF4E095E7FB0C94B52F93
:105C9000E92F0E94043058F3BA176207730784078C
:105CA000950720F079F4A6F50C9426300EF4E095D3
:105CB0000B2EBA2FA02D0B01B90190010C01CA01C6
:105CC000A0011124FF27591B99F0593F50F4503E71
:105CD00068F11A16F040A22F232F342F4427585F63
:105CE000F3CF469537952795A795F0405395C9F77B
:105CF0007EF41F16BA0B620B730B840BBAF0915033
:105D0000A1F0FF0FBB1F661F771F881FC2F70EC0D1
:105D1000BA0F621F731F841F48F4879577956795A4
:105D2000B795F7959E3F08F0B0CF9395880F08F090
:105D30009927EE0F9795879508950E94B12E0C94A0
:105D4000F32F0E94EC2F58F00E94E52F40F029F429
:105D50005F3F29F00C94B52F51110C9427300C940F
:105D6000BB2F0E94043068F39923B1F3552391F3BC
:105D7000951B550BBB27AA2762177307840738F0BA
:105D80009F5F5F4F220F331F441FAA1FA9F335D017
:105D90000E2E3AF0E0E832D091505040E695001CCB
:105DA000CAF72BD0FE2F29D0660F771F881FBB1F85
:105DB000261737074807AB07B0E809F0BB0B802D63
:105DC000BF01FF2793585F4F3AF09E3F510578F08F
:105DD0000C94B52F0C9427305F3FE4F3983ED4F336
:105DE000869577956795B795F7959F5FC9F7880F63
:105DF000911D9695879597F90895E1E0660F771FB5
:105E0000881FBB1F621773078407BA0720F0621B45
:105E1000730B840BBA0BEE1F88F7E095089529F4F5
:105E200016F00C94B52F0C9426300C94BB2F0E94C6
:105E30000C30A8F39638A0F707F80F92E8942BE3FC
:105E40003AEA48EB5FE70E94B9300F920F920F9247
:105E50004DB75EB70F920E946F30E8E5F1E00E9407
:105E6000BE2F4F915F91EF91FF91E595EE1FFF1FC0
:105E700049F0FE57E0684427EE0F441FFA95E1F71A
:105E80004195550B0E9439300F9007FE0C942D3030
:105E900008950E940C3088F09F5798F0B92F9927E9
:105EA000B751B0F0E1F0660F771F881F991F1AF005
:105EB000BA95C9F714C0B13091F00E942630B1E014
:105EC00008950C942630672F782F8827B85F39F013
:105ED000B93FCCF3869577956795B395D9F73EF49E
:105EE00090958095709561957F4F8F4F9F4F089546
:105EF000E89409C097FB3EF4909580957095619564
:105F00007F4F8F4F9F4F9923A9F0F92F96E9BB2719
:105F10009395F695879577956795B795F111F8CF95
:105F2000FAF4BB0F11F460FF1BC06F5F7F4F8F4F00
:105F30009F4F16C0882311F096E911C0772321F0F6
:105F40009EE8872F762F05C0662371F096E8862F8E
:105F500070E060E02AF09A95660F771F881FDAF7E5
:105F6000880F9695879597F9089597F99F6780E828
:105F700070E060E008959FEF80EC0895DF93CF9389
:105F80001F930F93FF92EF92DF927B018C01689435
:105F900006C0DA2EEF010E94B630FE01E894A5910A
:105FA0002591359145915591A6F3EF010E94482E18
:105FB000FE019701A801DA9469F7DF90EF90FF9056
:105FC0000F911F91CF91DF91089500240A94161626
:105FD000170618060906089500240A9412161306D7
:105FE000140605060895092E0394000C11F4882365
:105FF00052F0BB0F40F4BF2B11F460FF04C06F5F81
:106000007F4F8F4F9F4F089557FD9058440F551F56
:1060100059F05F3F71F04795880F97FB991F61F02A
:106020009F3F79F087950895121613061406551FA1
:10603000F2CF4695F1DF08C0161617061806991F0D
:10604000F1CF86957105610508940895E894BB2702
:1060500066277727CB0197F908959B01AC0160E093
:1060600070E080E89FE30C949D2E0C94B52F0C9467
:1060700018310E940C30D8F39923C9F3940F511DA5
:10608000A3F39150504094F059F0882332F0660FFA
:10609000771F881F91505040C1F79E3F51052CF744
:1060A000880F911D9695879597F908955F3FACF0FD
:1060B000983E9CF0BB27869577956795B79508F431
:1060C000B1609395C1F7BB0F58F711F460FFE8CFAB
:1060D0006F5F7F4F8F4F9F4FE3CF0C942730FA01B4
:1060E000DC01AA0FBB1F9B01AC01BF5728F422277C
:1060F00033274427507820C0B75190F4AB2F0024A9
:10610000469537952795011CA395D2F3002071F091
:10611000220F331F441FB395DAF30ED00C94302EA8
:1061200061307105A0E88A07B94630F49B01AC01E3
:106130006627772788279078309621F0208331834F
:106140004283538308950E94B6300C94F32F0E942B
:10615000E52F38F00E94EC2F20F0952311F00C94DD
:10616000B52F0C94BB2F11240C9427300E940430BF
:1061700070F3959FC1F3950F50E0551F629FF0019A
:10618000729FBB27F00DB11D639FAA27F00DB11DB3
:10619000AA1F649F6627B00DA11D661F829F22273C
:1061A000B00DA11D621F739FB00DA11D621F839FC3
:1061B000A00D611D221F749F3327A00D611D231F99
:1061C000849F600D211D822F762F6A2F11249F57E7
:1061D00050409AF0F1F088234AF0EE0FFF1FBB1FEA
:1061E000661F771F881F91505040A9F79E3F5105A9
:1061F00080F00C94B52F0C9427305F3FE4F3983E69
:10620000D4F3869577956795B795F795E7959F5F52
:10621000C1F7FE2B880F911D9695879597F90895E4
:106220009F930E9428310F9007FCEE5F0C94513130
:106230009F3F31F0915020F4879577956795B795FA
:10624000880F911D9695879597F908950C94BB2F0B
:106250000E940C30D8F3E894E0E0BB279F57F0F0A1
:106260002AED3FE049EC06C0EE0FBB0F661F771F1B
:10627000881F28F0B23A62077307840728F0B25AE1
:10628000620B730B840BE3959A9572F7803830F4A8
:106290009A95BB0F661F771F881FD2F790480C9402
:1062A0001A31EF93E0FF07C0A2EA2AED3FE049EC84
:1062B0005FEB0E94482E0E94F32F0F90039401FC85
:1062C0009058E0E8F1E00C9465319F938F937F93B1
:1062D0006F93FF93EF939B01AC010E94A330EF916A
:1062E000FF910E94BE2F2F913F914F915F910C948F
:1062F000A330AA1BBB1B51E107C0AA1FBB1FA617D7
:10630000B70710F0A61BB70B881F991F5A95A9F75E
:1063100080959095BC01CD01089597FB072E16F44A
:10632000009407D077FD09D00E94793107FC05D091
:106330003EF4909581959F4F0895709561957F4F9C
:106340000895EE0FFF1F0590F491E02D0994F9993F
:10635000FECF92BD81BDF89A992780B50895A6E138
:10636000B0E044E050E00C94E131A8E1B0E042E05C
:1063700050E00C94E131262FF999FECF92BD81BDFA
:10638000F89A019700B4021639F01FBA20BD0FB673
:10639000F894FA9AF99A0FBE08950396272F0E944F
:1063A000BC310E94BB31252F0E94BC31242F0C949C
:1063B000BC310196272F0E94BC310C94BB31DC010B
:1063C000CB01FC01F999FECF06C0F2BDE1BDF89A00
:1063D000319600B40D9241505040B8F70895F894AA
:0263E000FFCFED
:1063E2002001020C0328083C07140427A227772760
:1063F2004127072701000D010D020D030D040D05B4
:106402000D000C010C020C030C040C050C000B011A
:106412000B020B030B040B050B000A010A020A0311
:106422000A040A050A000901090209030904090507
:10643200090008010802080308040805080007010A
:106442000702070307040705070006010602060301
:1064520006040605060005010502050305040505F7
:1064620005000401040204030404040504000301FA
:1064720003020303030403050300020102020203F1
:1064820002040205020001010102010301040105E7
:1064920001000001000200030004000500010203E4
:1064A20004050607080900404D36393508E807B2E9
:0C64B2000779070C0725073E0757070075
:00000001FF
